:020000040000FA
:100000000228090083120313A001A101A2011230EA
:10001000A0003430A1005630A200B101B201B301FA
:10002000B401B501B601B701B801A401A3012C3098
:10003000A5000130A600A701A801AC01AC148530D1
:10004000A900850186018701831606309F0038309C
:100050008500860187010C10831201309000210871
:10006000B921AF00AF0E2108A721AF042C08AD00C5
:100070002C0CAD05AC182D13050DAD062D1BAF15C1
:1000800043282218AF150430B0009B202108882196
:10009000AF000230B0009B2020088821F039AF006B
:1000A0002008B921AF040130B0009B202F2885190A
:1000B0007E20051A6B20A20A0F3022050A3C031984
:1000C000622808001030A207F030A205603022023A
:1000D00003196B2808003F30AC05A201A10A0F30BC
:1000E00021050A3C0319752808001030A107F030DB
:1000F000A1056030210203197E2808002C1AA20AEB
:100100002C122C1D8A282C110830AC06AC19A00A20
:10011000AC1DA003A101A00A0F3020050A3C031961
:100120009628243020020319A00108001030A007EF
:10013000F030A00508002908A7070318A80A803096
:10014000A7070318A80A0C30A8072808AD000E0856
:100150002702031CAD030F08AD02AD1FA528F83020
:1001600085052F08860030088504FF30851E003085
:100170002C060139031DCA20A30A0319A40A260864
:100180002402031D080025082302031D08007F2107
:10019000572008002B082402AE002A082302031C63
:1001A000AE03AD002C1CEB282C102E08031D1429C7
:1001B0002D084B3C031C14290A302D02031C142962
:1001C00028302D02B10CB20CB30CB40CB50CB60C2B
:1001D000B70CB80C08002C142E0803190029023C97
:1001E000031C1429AE1C0029AC1C1A21B101B20158
:1001F000B301B401B501B601B701B801B117AC1034
:1002000024082602AE0023082502031CAE03AD001D
:100210002E08031D11292D08963C031C1129AC1C26
:100220005720AC1C7F211529AC142308AA002408F0
:10023000AB000800103038063F39031D0800B51C1C
:1002400008002C11B61A2C15C0303605403A031997
:10025000AC15C03A0319AC112C1235182C16340CFD
:10026000AE00350CAD00AE0CAD0C2D08AE00AE0CE2
:10027000AE062E08AE0CAE0CAE062E08AE0CAE0CC2
:10028000AE0CAE0CAE062E1855292D080F39093CC0
:10029000031C55292D087039503C031C55292D0885
:1002A0007F39A100A2017F212C17330C340CAD0043
:1002B0002D0C7F39AD00AE00AE00AE0CAE062E08A0
:1002C000AE0CAE0CAE062E08AE0CAE0CAE0CAE0CE8
:1002D000AE062E187E292D080F39093C031C7E29F5
:1002E0002D083039203C031C7E292D083F39233C42
:1002F000031C7E292D083F39A000AC1708000130EF
:100300002407A6002C3023070318A60AA50008001E
:10031000093C043C83189A29053EF039031900343E
:10032000103A0319C034303A0319F034103A031963
:10033000FC34FF34F03903198034103A0319E034E7
:10034000303A0319F834103A0319FE34FF34093CEB
:10035000043C8318B129053EF039503A031906349C
:100360000034F039403A03190434103A03190734C1
:1003700000340F3903190034013A03190834033AE1
:1003800003190C34013A03190E34073A03190F34D8
:10039000013A03190034033A03190834013A0319E6
:0A03A0000C340F3A03190E340F3429
:02400E00393B3C
:00000001FF
